 i2csdk

 Timestamp is 4da2a50a (Mon Apr 11 18:51:54 2011)

 Preferred load address is 10000000

 Start         Length     Name                   Class
 0001:00000000 00000004H .CRT$XCA                CODE
 0001:00000004 00000004H .CRT$XCZ                CODE
 0001:00000008 00000004H .CRT$XIA                CODE
 0001:0000000c 00000004H .CRT$XIZ                CODE
 0001:00000010 00000004H .CRT$XPA                CODE
 0001:00000014 00000004H .CRT$XPZ                CODE
 0001:00000018 00000004H .CRT$XTA                CODE
 0001:0000001c 00000004H .CRT$XTZ                CODE
 0001:00000020 000008c8H .rdata                  CODE
 0001:000008e8 00000023H .rdata$debug            CODE
 0001:0000090c 00001bd4H .text                   CODE
 0001:000024e0 00000014H .idata$2                CODE
 0001:000024f4 00000014H .idata$3                CODE
 0001:00002508 00000034H .idata$4                CODE
 0001:0000253c 0000000cH .idata$6                CODE
 0001:00002550 00000208H .edata                  CODE
 0002:00000000 00000034H .idata$5                DATA
 0002:00000038 0000044cH .data                   DATA
 0002:00000484 0000000cH .bss                    DATA
 0003:00000000 00000108H .pdata                  DATA

  Address         Publics by Value              Rva+Base       Lib:Object

 0000:00000000       ___safe_se_handler_table   00000000     <absolute>
 0000:00000000       ___safe_se_handler_count   00000000     <absolute>
 0001:00000000       __xc_a                     10001000     corelib0:crt0init.obj
 0001:00000004       __xc_z                     10001004     corelib0:crt0init.obj
 0001:00000008       __xi_a                     10001008     corelib0:crt0init.obj
 0001:0000000c       __xi_z                     1000100c     corelib0:crt0init.obj
 0001:00000010       __xp_a                     10001010     corelib0:crt0init.obj
 0001:00000014       __xp_z                     10001014     corelib0:crt0init.obj
 0001:00000018       __xt_a                     10001018     corelib0:crt0init.obj
 0001:0000001c       __xt_z                     1000101c     corelib0:crt0init.obj
 0001:0000003c       ??_C@_1O@IKMMPJPA@?$AA?9?$AA?9?$AA?$CF?$AAs?$AA?$AN?$AA?6?$AA?$AA@ 1000103c     i2csdk_common_topaz_v1:i2csdk.obj
 0001:0000004c       ??_C@_1DM@ELJGOEII@?$AA?$CF?$AAs?$AA?3?$AA?5?$AA?5?$AAC?$AAr?$AAe?$AAa?$AAt?$AAe?$AAF?$AAi?$AAl?$AAe?$AA?5?$AAI?$AA2?$AAC?$AA?5?$AAf?$AAa?$AAi?$AAl?$AAe?$AAd?$AA?$CB?$AA?$AN?$AA?6?$AA?$AA@ 1000104c     i2csdk_common_topaz_v1:i2csdk.obj
 0001:00000088       ??_C@_1O@JNDDBHKG@?$AA?$CL?$AA?$CL?$AA?$CF?$AAs?$AA?$AN?$AA?6?$AA?$AA@ 10001088     i2csdk_common_topaz_v1:i2csdk.obj
 0001:00000098       ??_C@_1BM@LKFHAAIO@?$AAI?$AA2?$AAC?$AAO?$AAp?$AAe?$AAn?$AAH?$AAa?$AAn?$AAd?$AAl?$AAe?$AA?$AA@ 10001098     i2csdk_common_topaz_v1:i2csdk.obj
 0001:000000b4       ??_C@_1DE@BBBAGJCD@?$AA?$CF?$AAs?$AA?3?$AA?5?$AAC?$AAl?$AAo?$AAs?$AAe?$AAH?$AAa?$AAn?$AAd?$AAl?$AAe?$AA?5?$AAf?$AAa?$AAi?$AAl?$AAe?$AAd?$AA?$CB?$AA?$AN?$AA?6?$AA?$AA@ 100010b4     i2csdk_common_topaz_v1:i2csdk.obj
 0001:000000e8       ??_C@_1BO@DIOAJNLH@?$AAI?$AA2?$AAC?$AAC?$AAl?$AAo?$AAs?$AAe?$AAH?$AAa?$AAn?$AAd?$AAl?$AAe?$AA?$AA@ 100010e8     i2csdk_common_topaz_v1:i2csdk.obj
 0001:00000108       ??_C@_1EO@NIIMKOHH@?$AA?$CF?$AAs?$AA?3?$AA?5?$AAI?$AA2?$AAC?$AA_?$AAI?$AAO?$AAC?$AAT?$AAL?$AA_?$AAS?$AAE?$AAT?$AA_?$AAS?$AAL?$AAA?$AAV?$AAE?$AA_?$AAM?$AAO?$AAD?$AAE?$AA?5?$AAf?$AAa?$AAi@ 10001108     i2csdk_common_topaz_v1:i2csdk.obj
 0001:00000158       ??_C@_1CA@FFLJNIAM@?$AAI?$AA2?$AAC?$AAS?$AAe?$AAt?$AAS?$AAl?$AAa?$AAv?$AAe?$AAM?$AAo?$AAd?$AAe?$AA?$AA@ 10001158     i2csdk_common_topaz_v1:i2csdk.obj
 0001:00000178       ??_C@_1FA@HBGKOJOG@?$AA?$CF?$AAs?$AA?3?$AA?5?$AAI?$AA2?$AAC?$AA_?$AAI?$AAO?$AAC?$AAT?$AAL?$AA_?$AAS?$AAE?$AAT?$AA_?$AAM?$AAA?$AAS?$AAT?$AAE?$AAR?$AA_?$AAM?$AAO?$AAD?$AAE?$AA?5?$AAf?$AAa@ 10001178     i2csdk_common_topaz_v1:i2csdk.obj
 0001:000001c8       ??_C@_1CC@OLKFNAJN@?$AAI?$AA2?$AAC?$AAS?$AAe?$AAt?$AAM?$AAa?$AAs?$AAt?$AAe?$AAr?$AAM?$AAo?$AAd?$AAe?$AA?$AA@ 100011c8     i2csdk_common_topaz_v1:i2csdk.obj
 0001:000001f0       ??_C@_1EE@OGCLBJC@?$AA?$CF?$AAs?$AA?3?$AA?5?$AAI?$AA2?$AAC?$AA_?$AAI?$AAO?$AAC?$AAT?$AAL?$AA_?$AAI?$AAS?$AA_?$AAM?$AAA?$AAS?$AAT?$AAE?$AAR?$AA?5?$AAf?$AAa?$AAi?$AAl?$AAe?$AAd?$AA?$CB?$AA?$AN@ 100011f0     i2csdk_common_topaz_v1:i2csdk.obj
 0001:00000234       ??_C@_1BI@OBFMPFIJ@?$AAI?$AA2?$AAC?$AAI?$AAs?$AAM?$AAa?$AAs?$AAt?$AAe?$AAr?$AA?$AA@ 10001234     i2csdk_common_topaz_v1:i2csdk.obj
 0001:00000250       ??_C@_1EC@HGOOCBEA@?$AA?$CF?$AAs?$AA?3?$AA?5?$AAI?$AA2?$AAC?$AA_?$AAI?$AAO?$AAC?$AAT?$AAL?$AA_?$AAI?$AAS?$AA_?$AAS?$AAL?$AAA?$AAV?$AAE?$AA?5?$AAf?$AAa?$AAi?$AAl?$AAe?$AAd?$AA?$CB?$AA?$AN?$AA?6@ 10001250     i2csdk_common_topaz_v1:i2csdk.obj
 0001:00000294       ??_C@_1BG@HLPLEEMI@?$AAI?$AA2?$AAC?$AAI?$AAs?$AAS?$AAl?$AAa?$AAv?$AAe?$AA?$AA@ 10001294     i2csdk_common_topaz_v1:i2csdk.obj
 0001:000002b0       ??_C@_1EO@IDIGFDOF@?$AA?$CF?$AAs?$AA?3?$AA?5?$AAI?$AA2?$AAC?$AA_?$AAI?$AAO?$AAC?$AAT?$AAL?$AA_?$AAG?$AAE?$AAT?$AA_?$AAC?$AAL?$AAO?$AAC?$AAK?$AA_?$AAR?$AAA?$AAT?$AAE?$AA?5?$AAf?$AAa?$AAi@ 100012b0     i2csdk_common_topaz_v1:i2csdk.obj
 0001:00000300       ??_C@_1CA@NOOCADPH@?$AAI?$AA2?$AAC?$AAG?$AAe?$AAt?$AAC?$AAl?$AAo?$AAc?$AAk?$AAR?$AAa?$AAt?$AAe?$AA?$AA@ 10001300     i2csdk_common_topaz_v1:i2csdk.obj
 0001:00000320       ??_C@_1EO@NAPNIMLP@?$AA?$CF?$AAs?$AA?3?$AA?5?$AAI?$AA2?$AAC?$AA_?$AAI?$AAO?$AAC?$AAT?$AAL?$AA_?$AAS?$AAE?$AAT?$AA_?$AAC?$AAL?$AAO?$AAC?$AAK?$AA_?$AAR?$AAA?$AAT?$AAE?$AA?5?$AAf?$AAa?$AAi@ 10001320     i2csdk_common_topaz_v1:i2csdk.obj
 0001:00000370       ??_C@_1CA@FOCEMOFB@?$AAI?$AA2?$AAC?$AAS?$AAe?$AAt?$AAC?$AAl?$AAo?$AAc?$AAk?$AAR?$AAa?$AAt?$AAe?$AA?$AA@ 10001370     i2csdk_common_topaz_v1:i2csdk.obj
 0001:00000390       ??_C@_1EM@FBDMNHMP@?$AA?$CF?$AAs?$AA?3?$AA?5?$AAI?$AA2?$AAC?$AA_?$AAI?$AAO?$AAC?$AAT?$AAL?$AA_?$AAS?$AAE?$AAT?$AA_?$AAF?$AAR?$AAE?$AAQ?$AAU?$AAE?$AAN?$AAC?$AAY?$AA?5?$AAf?$AAa?$AAi?$AAl@ 10001390     i2csdk_common_topaz_v1:i2csdk.obj
 0001:000003dc       ??_C@_1CA@IDHFHNDJ@?$AAI?$AA2?$AAC?$AAS?$AAe?$AAt?$AAF?$AAr?$AAe?$AAq?$AAu?$AAe?$AAn?$AAc?$AAy?$AA?$AA@ 100013dc     i2csdk_common_topaz_v1:i2csdk.obj
 0001:00000400       ??_C@_1EM@DAFLIJHB@?$AA?$CF?$AAs?$AA?3?$AA?5?$AAI?$AA2?$AAC?$AA_?$AAI?$AAO?$AAC?$AAT?$AAL?$AA_?$AAS?$AAE?$AAT?$AA_?$AAS?$AAE?$AAL?$AAF?$AA_?$AAA?$AAD?$AAD?$AAR?$AA?5?$AAf?$AAa?$AAi?$AAl@ 10001400     i2csdk_common_topaz_v1:i2csdk.obj
 0001:0000044c       ??_C@_1BO@FJIJIDHN@?$AAI?$AA2?$AAC?$AAS?$AAe?$AAt?$AAS?$AAe?$AAl?$AAf?$AAA?$AAd?$AAd?$AAr?$AA?$AA@ 1000144c     i2csdk_common_topaz_v1:i2csdk.obj
 0001:00000470       ??_C@_1EM@DOOMHNIK@?$AA?$CF?$AAs?$AA?3?$AA?5?$AAI?$AA2?$AAC?$AA_?$AAI?$AAO?$AAC?$AAT?$AAL?$AA_?$AAG?$AAE?$AAT?$AA_?$AAS?$AAE?$AAL?$AAF?$AA_?$AAA?$AAD?$AAR?$AAR?$AA?5?$AAf?$AAa?$AAi?$AAl@ 10001470     i2csdk_common_topaz_v1:i2csdk.obj
 0001:000004bc       ??_C@_1BO@EPOEGCBP@?$AAI?$AA2?$AAC?$AAG?$AAe?$AAt?$AAS?$AAe?$AAl?$AAf?$AAA?$AAd?$AAd?$AAr?$AA?$AA@ 100014bc     i2csdk_common_topaz_v1:i2csdk.obj
 0001:000004e0       ??_C@_1EC@KHHHEPPO@?$AA?$CF?$AAs?$AA?3?$AA?5?$AAI?$AA2?$AAC?$AA_?$AAI?$AAO?$AAC?$AAT?$AAL?$AA_?$AAT?$AAR?$AAA?$AAN?$AAS?$AAF?$AAE?$AAR?$AA?5?$AAf?$AAa?$AAi?$AAl?$AAe?$AAd?$AA?$CB?$AA?$AN?$AA?6@ 100014e0     i2csdk_common_topaz_v1:i2csdk.obj
 0001:00000524       ??_C@_1BI@DJKHLHDJ@?$AAI?$AA2?$AAC?$AAT?$AAr?$AAa?$AAn?$AAs?$AAf?$AAe?$AAr?$AA?$AA@ 10001524     i2csdk_common_topaz_v1:i2csdk.obj
 0001:0000053c       ??_C@_1DM@JKNKIGKG@?$AA?$CF?$AAs?$AA?3?$AA?5?$AAI?$AA2?$AAC?$AA_?$AAI?$AAO?$AAC?$AAT?$AAL?$AA_?$AAR?$AAE?$AAS?$AAE?$AAT?$AA?5?$AAf?$AAa?$AAi?$AAl?$AAe?$AAd?$AA?$CB?$AA?$AN?$AA?6?$AA?$AA@ 1000153c     i2csdk_common_topaz_v1:i2csdk.obj
 0001:00000578       ??_C@_1BC@OIDPNOGD@?$AAI?$AA2?$AAC?$AAR?$AAe?$AAs?$AAe?$AAt?$AA?$AA@ 10001578     i2csdk_common_topaz_v1:i2csdk.obj
 0001:00000590       ??_C@_1EK@MBLCGJPN@?$AA?$CF?$AAs?$AA?3?$AA?5?$AAI?$AA2?$AAC?$AA_?$AAI?$AAO?$AAC?$AAT?$AAL?$AA_?$AAE?$AAN?$AAA?$AAB?$AAL?$AAE?$AA_?$AAS?$AAL?$AAA?$AAV?$AAE?$AA?5?$AAf?$AAa?$AAi?$AAl?$AAe@ 10001590     i2csdk_common_topaz_v1:i2csdk.obj
 0001:000005dc       ??_C@_1BO@MPCLPGJL@?$AAI?$AA2?$AAC?$AAE?$AAn?$AAa?$AAb?$AAl?$AAe?$AAS?$AAl?$AAa?$AAv?$AAe?$AA?$AA@ 100015dc     i2csdk_common_topaz_v1:i2csdk.obj
 0001:00000600       ??_C@_1EM@NGIGKOFA@?$AA?$CF?$AAs?$AA?3?$AA?5?$AAI?$AA2?$AAC?$AA_?$AAI?$AAO?$AAC?$AAT?$AAL?$AA_?$AAD?$AAI?$AAS?$AAA?$AAB?$AAL?$AAE?$AA_?$AAS?$AAL?$AAA?$AAV?$AAE?$AA?5?$AAf?$AAa?$AAi?$AAl@ 10001600     i2csdk_common_topaz_v1:i2csdk.obj
 0001:0000064c       ??_C@_1CA@MDKFOKJO@?$AAI?$AA2?$AAC?$AAD?$AAi?$AAs?$AAa?$AAb?$AAl?$AAe?$AAS?$AAl?$AAa?$AAv?$AAe?$AA?$AA@ 1000164c     i2csdk_common_topaz_v1:i2csdk.obj
 0001:00000670       ??_C@_1EM@CDABHHLM@?$AA?$CF?$AAs?$AA?3?$AA?5?$AAI?$AA2?$AAC?$AA_?$AAI?$AAO?$AAC?$AAT?$AAL?$AA_?$AAG?$AAE?$AAT?$AA_?$AAS?$AAL?$AAA?$AAV?$AAE?$AAS?$AAI?$AAZ?$AAE?$AA?5?$AAf?$AAa?$AAi?$AAl@ 10001670     i2csdk_common_topaz_v1:i2csdk.obj
 0001:000006bc       ??_C@_1CA@BDKLMOJN@?$AAI?$AA2?$AAC?$AAG?$AAe?$AAt?$AAS?$AAl?$AAa?$AAv?$AAe?$AAS?$AAi?$AAz?$AAe?$AA?$AA@ 100016bc     i2csdk_common_topaz_v1:i2csdk.obj
 0001:000006e0       ??_C@_1EM@LIDKAFIO@?$AA?$CF?$AAs?$AA?3?$AA?5?$AAI?$AA2?$AAC?$AA_?$AAI?$AAO?$AAC?$AAT?$AAL?$AA_?$AAS?$AAE?$AAT?$AA_?$AAS?$AAL?$AAA?$AAV?$AAE?$AAS?$AAI?$AAZ?$AAE?$AA?5?$AAf?$AAa?$AAi?$AAl@ 100016e0     i2csdk_common_topaz_v1:i2csdk.obj
 0001:0000072c       ??_C@_1CA@JDGNADDL@?$AAI?$AA2?$AAC?$AAS?$AAe?$AAt?$AAS?$AAl?$AAa?$AAv?$AAe?$AAS?$AAi?$AAz?$AAe?$AA?$AA@ 1000172c     i2csdk_common_topaz_v1:i2csdk.obj
 0001:00000750       ??_C@_1EM@BAGCIELJ@?$AA?$CF?$AAs?$AA?3?$AA?5?$AAI?$AA2?$AAC?$AA_?$AAI?$AAO?$AAC?$AAT?$AAL?$AA_?$AAG?$AAE?$AAT?$AA_?$AAS?$AAL?$AAA?$AAV?$AAE?$AA_?$AAT?$AAX?$AAT?$AA?5?$AAf?$AAa?$AAi?$AAl@ 10001750     i2csdk_common_topaz_v1:i2csdk.obj
 0001:0000079c       ??_C@_1CA@DLFFBFK@?$AAI?$AA2?$AAC?$AAG?$AAe?$AAt?$AAS?$AAl?$AAa?$AAv?$AAe?$AAT?$AAe?$AAx?$AAt?$AA?$AA@ 1000179c     i2csdk_common_topaz_v1:i2csdk.obj
 0001:000007c0       ??_C@_1EM@ILFJPGIL@?$AA?$CF?$AAs?$AA?3?$AA?5?$AAI?$AA2?$AAC?$AA_?$AAI?$AAO?$AAC?$AAT?$AAL?$AA_?$AAS?$AAE?$AAT?$AA_?$AAS?$AAL?$AAA?$AAV?$AAE?$AA_?$AAT?$AAX?$AAT?$AA?5?$AAf?$AAa?$AAi?$AAl@ 100017c0     i2csdk_common_topaz_v1:i2csdk.obj
 0001:0000080c       ??_C@_1CA@IDHDJMPM@?$AAI?$AA2?$AAC?$AAS?$AAe?$AAt?$AAS?$AAl?$AAa?$AAv?$AAe?$AAT?$AAe?$AAx?$AAt?$AA?$AA@ 1000180c     i2csdk_common_topaz_v1:i2csdk.obj
 0001:00000830       ??_C@_1FM@ECAKLGED@?$AA?$CK?$AA?$CK?$AA?$CK?$AA?$CK?$AA?$CK?$AA?5?$AAD?$AAL?$AAL?$AA?5?$AAP?$AAR?$AAO?$AAC?$AAE?$AAS?$AAS?$AA?5?$AAD?$AAE?$AAT?$AAA?$AAC?$AAH?$AA?5?$AAF?$AAR?$AAO?$AAM?$AA?5?$AAI?$AA2@ 10001830     i2csdk_common_topaz_v1:i2csdk.obj
 0001:00000890       ??_C@_1FI@FDMCCIJN@?$AA?$CK?$AA?$CK?$AA?$CK?$AA?$CK?$AA?$CK?$AA?5?$AAD?$AAL?$AAL?$AA?5?$AAP?$AAR?$AAO?$AAC?$AAE?$AAS?$AAS?$AA?5?$AAA?$AAT?$AAT?$AAA?$AAC?$AAH?$AA?5?$AAT?$AAO?$AA?5?$AAI?$AA2?$AAC?$AA?5@ 10001890     i2csdk_common_topaz_v1:i2csdk.obj
 0001:0000090c       I2COpenHandle              1000190c f   i2csdk_common_topaz_v1:i2csdk.obj
 0001:00000a24       I2CCloseHandle             10001a24 f   i2csdk_common_topaz_v1:i2csdk.obj
 0001:00000b1c       I2CSetSlaveMode            10001b1c f   i2csdk_common_topaz_v1:i2csdk.obj
 0001:00000c38       I2CSetMasterMode           10001c38 f   i2csdk_common_topaz_v1:i2csdk.obj
 0001:00000d54       I2CIsMaster                10001d54 f   i2csdk_common_topaz_v1:i2csdk.obj
 0001:00000e70       I2CIsSlave                 10001e70 f   i2csdk_common_topaz_v1:i2csdk.obj
 0001:00000f8c       I2CGetClockRate            10001f8c f   i2csdk_common_topaz_v1:i2csdk.obj
 0001:000010a8       I2CSetClockRate            100020a8 f   i2csdk_common_topaz_v1:i2csdk.obj
 0001:000011c4       I2CSetFrequency            100021c4 f   i2csdk_common_topaz_v1:i2csdk.obj
 0001:000012e0       I2CSetSelfAddr             100022e0 f   i2csdk_common_topaz_v1:i2csdk.obj
 0001:000013fc       I2CGetSelfAddr             100023fc f   i2csdk_common_topaz_v1:i2csdk.obj
 0001:00001518       I2CTransfer                10002518 f   i2csdk_common_topaz_v1:i2csdk.obj
 0001:00001634       I2CReset                   10002634 f   i2csdk_common_topaz_v1:i2csdk.obj
 0001:00001750       I2CEnableSlave             10002750 f   i2csdk_common_topaz_v1:i2csdk.obj
 0001:0000186c       I2CDisableSlave            1000286c f   i2csdk_common_topaz_v1:i2csdk.obj
 0001:00001988       I2CGetSlaveSize            10002988 f   i2csdk_common_topaz_v1:i2csdk.obj
 0001:00001aa4       I2CSetSlaveSize            10002aa4 f   i2csdk_common_topaz_v1:i2csdk.obj
 0001:00001bc0       I2CGetSlaveText            10002bc0 f   i2csdk_common_topaz_v1:i2csdk.obj
 0001:00001cdc       I2CSetSlaveText            10002cdc f   i2csdk_common_topaz_v1:i2csdk.obj
 0001:00001df8       DllEntry                   10002df8 f   i2csdk_common_topaz_v1:i2csdk.obj
 0001:00001ebc       CreateFileW                10002ebc f   coredll:COREDLL.dll
 0001:00001ecc       NKDbgPrintfW               10002ecc f   coredll:COREDLL.dll
 0001:00001edc       CloseHandle                10002edc f   coredll:COREDLL.dll
 0001:00001eec       DeviceIoControl            10002eec f   coredll:COREDLL.dll
 0001:00001efc       DisableThreadLibraryCalls  10002efc f   coredll:COREDLL.dll
 0001:00001f0c       RegisterDbgZones           10002f0c f   coredll:COREDLL.dll
 0001:00001f1c       _DllEntryCRTStartup        10002f1c f   corelib0:pegdentry.obj
 0001:00001f88       exit                       10002f88 f   corelib0:cexit.obj
 0001:000020ac       _exit                      100030ac f   corelib0:cexit.obj
 0001:000020cc       _cexit                     100030cc f   corelib0:cexit.obj
 0001:000020e4       _c_exit                    100030e4 f   corelib0:cexit.obj
 0001:000020fc       _initterm                  100030fc f   corelib0:crt0dat.obj
 0001:00002148       _cinit                     10003148 f   corelib0:crt0dat.obj
 0001:00002178       __security_init_cookie     10003178 f   corelib0:seccinit.obj
 0001:00002210       __crt_ExitProcess          10003210 f   corelib0:exitproc_proxy.obj
 0001:0000223c       GetCurrentProcess          1000323c f i corelib0:exitproc_proxy.obj
 0001:00002254       _onexit                    10003254 f   corelib0:onexit.obj
 0001:00002430       atexit                     10003430 f   corelib0:onexit.obj
 0001:00002480       free                       10003480 f   corelib1:COREDLL.dll
 0001:00002490       __security_gen_cookie2     10003490 f   corelib1:COREDLL.dll
 0001:000024a0       realloc                    100034a0 f   corelib1:COREDLL.dll
 0001:000024b0       malloc                     100034b0 f   corelib1:COREDLL.dll
 0001:000024c0       _msize                     100034c0 f   corelib1:COREDLL.dll
 0001:000024d0       TerminateProcess           100034d0 f   coredll:COREDLL.dll
 0001:000024e0       __IMPORT_DESCRIPTOR_COREDLL 100034e0     coredll:COREDLL.dll
 0001:000024f4       __NULL_IMPORT_DESCRIPTOR   100034f4     coredll:COREDLL.dll
 0002:00000000       __imp_CreateFileW          10004000     coredll:COREDLL.dll
 0002:00000004       __imp_NKDbgPrintfW         10004004     coredll:COREDLL.dll
 0002:00000008       __imp_CloseHandle          10004008     coredll:COREDLL.dll
 0002:0000000c       __imp_DeviceIoControl      1000400c     coredll:COREDLL.dll
 0002:00000010       __imp_DisableThreadLibraryCalls 10004010     coredll:COREDLL.dll
 0002:00000014       __imp_RegisterDbgZones     10004014     coredll:COREDLL.dll
 0002:00000018       __imp_free                 10004018     corelib1:COREDLL.dll
 0002:0000001c       __imp___security_gen_cookie2 1000401c     corelib1:COREDLL.dll
 0002:00000020       __imp_realloc              10004020     corelib1:COREDLL.dll
 0002:00000024       __imp_malloc               10004024     corelib1:COREDLL.dll
 0002:00000028       __imp__msize               10004028     corelib1:COREDLL.dll
 0002:0000002c       __imp_TerminateProcess     1000402c     coredll:COREDLL.dll
 0002:00000030       \177COREDLL_NULL_THUNK_DATA 10004030     coredll:COREDLL.dll
 0002:00000038       dpCurSettings              10004038     i2csdk_common_topaz_v1:i2csdk.obj
 0002:0000047c       __security_cookie          1000447c     corelib0:seccinit.obj
 0002:00000480       __security_cookie_complement 10004480     corelib0:seccinit.obj
 0002:00000484       _exitflag                  10004484     corelib0:cexit.obj
 0002:00000488       __onexitend                10004488     <common>
 0002:0000048c       __onexitbegin              1000448c     <common>

 entry point at        0001:00001f1c

 Static symbols

 0001:00001fa8       doexit                     10002fa8 f   corelib0:cexit.obj
